:020000040000FA
:0600000007309F00962866
:08000800F1000308F20083017E
:100010008C10AD01F030850520302D0784000008DC
:100020004720AE00023003152D02031D1B287D3032
:100030002402031C2E152E0886002D08B6203C3005
:10004000AE00AE0B2128AD0A043003112D02031DB2
:100050000A280511A40AFA302402031D4228A4012B
:10006000A70A3C302702031D4228A701A60A3C30FC
:100070002602031D4228A601A50A18302502031DE9
:100080004228A50172088300F10E710E09000F3994
:1000900082077B344834D334DA34E834BA34BB349E
:1000A0005834FB34FA340034C220D2205920640082
:1000B0005428A80A7F30280203196328FF30280239
:1000C00003196728080005083039AB000800050847
:1000D00030392B06031D0800A90A2A082902031C2F
:1000E0000800A9010630AA002B1E7C28AB1E892817
:1000F0000130AA00AC0108002C08031D81280D3036
:10010000AA002C14A701A50A183025020319A5017D
:1001100008002C08031D8E280D30AA002C14A701FE
:10012000A60A3C3026020319A6010800640000302C
:10013000860085018316F03085000030860080300F
:100140008100F93092008C14831207309200203025
:100150008400A401A501A601A701A801A901AA0183
:10016000AB01AC0164000B178B1754288207BC2825
:10017000BE28C0280515C1288515C1288514C128A9
:1001800005140800AF012608B000F630B007AF0A2A
:100190000318C528AF032F08A1000A30B0073008A4
:1001A000A0000800AF012508B000F630B007AF0A84
:1001B0000318D528AF032F080A30031D2F08A3000A
:0A01C0000A30B0073008A200080062
:02400E00093F68
:00000001FF
